:020000040000FA
:020000006C286A
:080008008B13A300030EA400FA
:100010000C1C2A28D0308F00050804392C06031D3B
:100020001F28A80B29282C08AB00043A031D1A2806
:1000300085161B2885122708A800A90029288400F6
:10004000AC06A90B272885122B112708A900270821
:10005000A8000C100B1D37288B1E352825088100A1
:10006000851C34288510352885140B113728240E5B
:100070008300A30E230E8B170900831641308100E5
:100080000530850010309F000C14FF239000831270
:100090000F309F00073099008510851101309000C6
:1000A0008B160B178B1708004E30A5000030A600EA
:1000B0000030A6000030AC00AB001030A700A80054
:1000C000A9000800A20B6228080085160A306220E9
:1000D00085120A30622065283D20542005187328B7
:1000E0008B122610792826187928261425088100D5
:0400F0008B166E28D5
:00000001FF
